:020000040000FA
:100000000A128A116328820730343134323433348F
:100010003434353436343734383439344134423476
:1000200043344434453446341030B0000310A40D3A
:10003000A50D0310A00DA10D031C24282308A5075E
:100040002208A4070318A50AB00B162808002030C0
:10005000B000A401A501A601A7010310AC0DAD0DD0
:10006000AE0DAF0D0310A00DA10DA20DA30DA40D9B
:10007000A50DA60DA70D27082B02031D492826084C
:100080002A02031D492825082902031D492824089E
:10009000280203194D2803185C282808A4022908FF
:1000A000031C290FA5022A08031C2A0FA6022B08ED
:1000B000031C2B0FA7022C14B00B2D2808008A005C
:1000C0008312320882000608B90083169B0183124E
:1000D0009F0183169F0107309C008F300F057038F9
:1000E0008F00D9288316B0003008031908000130AA
:1000F0003002031D802800000000000000000800FE
:10010000B00300000000B1018F28831203130330F5
:10011000A0000A128A11A00B8B288316B10A31089D
:100120003002031D85280800AE01AF01A928831203
:1001300003130330A0008330A1000A128A11A10B1F
:100140009D280A128A11A00B9B288316AE0A031958
:10015000AF0A2E082C028312A00083162F082D024E
:1001600083122004031D97280800AA01AB01CD28A3
:1001700083120313B430A000DD30A1000A128A11EB
:10018000A10BBE280A128A11A00BBC280000000097
:1001900000008316AA0A0319AB0A2A082802831250
:1001A000A00083162B08290283122004031DB828FF
:1001B0000800831242104D292208A6002308A70038
:1001C0008312EF01F8288316240883126F07840036
:1001D000831383162518831700088312A000831643
:1001E00020088312B200831621085F208312EF0AD1
:1001F0006F08831626028312A00083162708831235
:100200002004031DE3280800EC00421C14293030B0
:10021000A0006A08B2006B085F2078308312A0004B
:100220006A08B2006B085F2083126C0E0F39ED0074
:100230000F306D05EE0000308A006E080320831237
:10024000A0006A08B2006B085F200F3083126C05B3
:10025000ED0000308A006D0803208312A0006A08B8
:10026000B2006B085F28CF3083169900181508007C
:10027000332183168C120C1298169030831298003A
:1002800008008312B8000C1E4329380899000800A2
:1002900083122008B7003708412938212130412135
:1002A0008A298312E9006908031D592983161B1442
:1002B0000514013083126902031D612983169B1402
:1002C0008514023083126902031D692983161B15E8
:1002D0000515033083126902031D712983169B15CE
:1002E0008515043083126902031D792983161B16B4
:1002F0000516053083126902031D812983169B169A
:100300000617063083126902031D892983161B17FD
:10031000861708008312C301430EA0003030A005E9
:10032000CF3083161F058312200483169F003A2ABC
:1003300068106408A0006508A1000A30A200A301AB
:10034000142083122408E6002508E7000310670C38
:10035000A100660CA0000310A10CA00C0310A10CBE
:10036000A00C2008BA0010303A02E810031D031850
:10037000E8143C303A0268110319C029031C6815BF
:10038000E815E818681DE811E819681420106818C5
:1003900020140800F8308312E2054030E400E50143
:1003A00098218312E2112018E215E21DDC29F830B1
:1003B00062050638E200242A2030E400E501982195
:1003C0008312E2122018E216E21EEB29F8306205D1
:1003D0000238E200242A1030E400E501982183125B
:1003E000E2132018E217E21FFA29F83062050538F7
:1003F000E200242A0830E400E50198218312E3108A
:100400002018E314E31C092AF83062050138E200E1
:10041000242A0430E400E50198218312E311201816
:10042000E315E31D182AF83062050438E200242A97
:100430000230E400E50198218312E3122018E3164C
:10044000E31E242AF830E20503306205A000200CE8
:10045000A100A10C210CA100C030A1053F301F0557
:1004600021049F006219372A83161F130800831680
:100470001F1708008312B401802AE000600DA0005D
:10048000A00DA00D3830A005C7301F0520049F0027
:100490001F143B08722083121F151F194D2A1E08B6
:1004A000E10026303A020319572A031C612A8312FD
:1004B00003134E30A0000A128A11A00B5D2A00001F
:1004C0006B2A831203131330A0000A128A11A00BA7
:1004D000672A000000001F10610808008312DE0078
:1004E0005E083D228312DF005F08080083169F1319
:1004F000080015308312BB0008007622CA21792A31
:100500007D22043051218312B5010130B600ED2A5D
:100510005708A8005808A9005908AA005A08AB00B3
:10052000A0011230A1007A30A200A301272083127B
:100530002C08DB002D08DC0003105C0CB6005B0C03
:10054000B5000310B60CB50C9201350836045D14E5
:1005500003195D1010303602031DB02A0030350239
:10056000DD10031D031CDD145D155D18DD1C5D1120
:100570005D1DEC2A01303602031DC02A0030350211
:100580000319C42A0318C72AFC309205E72A04304D
:100590003602031DCD2A003035020319D12A031873
:1005A000DC2A0310B60CB50C0310B60CB50CFC30ED
:1005B000120501389200E72A0430A0000310B60C9F
:1005C000B50CA00BDE2AFC30120502389200350370
:1005D00083169200831212150800BC01BD01702B16
:1005E000F0303D050C38BD003C0895003D089700F3
:1005F0000800F0308312BD053D0897000800033065
:100600005602031D052BFF30550203190D2B031C49
:100610000D2BFF30D5000330D6000310560CA1007F
:10062000550CA0000310A10CA00C2008BC00033046
:100630005505A000200EA1003030A105CF303D05AA
:100640002104BD00F02A8312CC004C08031D2B2B83
:10065000CD01CE01632B64304C020319312B031CF6
:10066000392B3608CE003503CD004D0A0319CE03D1
:10067000632B4C08CF00D0010310360CD200350C90
:10068000D1000310D20CD10C4F08A0005008A100DB
:100690005108A2005208A300142083122408D3009A
:1006A0002508D4001930A800A901AA01AB015308FC
:1006B000A0005408A100A201A301272083122C0846
:1006C000CD002D08CE0003104D0DCF004E0DD000F3
:1006D0000310CF0DD00D4F08D5005008D600FF2ACB
:1006E0008316061086130D308312BF000A30C00037
:1006F000C2104215C101B91339088600D62BF02269
:10070000F4308312D7000130D800D901DA018822F1
:100710003230232301308316A800A901B520F92A1D
:10072000F0228312C401C501C601C7014408C800F4
:100730004508C9004608CA004708CB00F430C8077E
:100740000130FE0003187E0FC9070030FE000318B9
:100750007E0FCA070030FE0003187E0FCB07480843
:10076000D7004908D8004A08D9004B08DA00882287
:10077000323023230A308316AC00AD01942083125B
:10078000C40A0319C50A0319C60A0319C70AF430B3
:100790004402A00001304502A00400304602A0043B
:1007A000003047022004031D962BF92A04306E22E4
:1007B0008312BE0020303E020319E72B031CE72BF7
:1007C000C214421DE82B902383124211E82BC21061
:1007D000C21CF82BB91739088600C10A053041023E
:1007E0000319F92B031CF92B7F238312C101F92B69
:1007F000C1014830EA000130EB003E0804214830D6
:100800008316A0000130A1000230A200A3013F30F6
:10081000A400A501DC200A308316A800A901B52098
:02082000D62BD5
:02400E00F83F79
:02401000FF3F70
:00000001FF
